:1000000010C022C021C020C01FC01EC01DC01CC007
:100010001BC01AC019C018C017C016C015C014C024
:1000200013C011241FBECFE5D2E0DEBFCDBF12E06A
:10003000A0E6B0E0ECEFF5E002C005900D92AE381E
:10004000B107D9F72BD1D8C2DBCF81E08A95F1F780
:1000500008958AEF90E00197F1F708958F929F92AB
:10006000AF92BF92CF92DF92EF92FF92BC0180E0FD
:1000700090E090D14B015C0120E030E04AE753E48E
:1000800017D26B017C0120E030E040E85FE352D101
:1000900087FD20C020E03FEF4FE757E4C701B601DE
:1000A00003D218169CF420E030E040E251E4C50190
:1000B000B401FED143D129E130E06115710579F039
:1000C000C9010197F1F761507109F7CFC701B60176
:1000D00035D102C061E070E0CB010197F1F7FF90EC
:1000E000EF90DF90CF90BF90AF909F908F9008954A
:1000F000DB98611102C0DA9801C0DA9A98E087FFB4
:1001000002C0D99A01C0D998D898880FD89A91502E
:10011000B1F7DB9A0895CF93DF9360E08CE0E8DFDE
:1001200060E080E8E5DFC8EFD1E061E080E0E0DF9B
:100130002197D9F7DF91CF9108958AB38F618ABB58
:10014000DC9883DFDC9ADB9880DFDB9A7EDF60E07F
:1001500081E2CEDF60E088ECCBDF60E086E0C8DFE4
:1001600060E083E1C5DF60E080E2C2DFD4DF60E011
:100170008CE0BEDFDB980895CF93C82F862F60E018
:100180008064B6DF60E08C2F8068CF91B1CF0F9391
:100190001F93CF93DF93805290E066E070E01BD214
:1001A0008C01005A1F4FC0E0D0E0F801EC0FFD1F9A
:1001B00061E080819DDF2196C630D105B1F7DF91E6
:1001C000CF911F910F9108950F931F93CF93DF93BA
:1001D00000D0CDB7DEB749835A83CEDF4981042FE3
:1001E0005A81152FF80181918F01882311F0CFDFFB
:1001F000F9CF0F900F90DF91CF911F910F9108953C
:100200006F927F928F929F92AF92BF92CF92DF9226
:10021000EF92FF920F931F93CF93DF93682E762E6A
:10022000802F877006950695069581110F5FC22E67
:10023000D12CEA01AA24BB24A41AB50AE12CF12C82
:1002400010E0672D6E0DE016F106B8F4862D94DFF0
:100250004E0194012A0D3B1D2C153D0530F461E043
:10026000F40181914F0144DFF4CFFFEFEF1AFF0A51
:10027000CC0DDD1DAC18BD08E4CFDF91CF911F91EF
:100280000F91FF90EF90DF90CF90BF90AF909F9035
:100290008F907F906F9008950895089581E087BBB7
:1002A0008FE18ABB4ADF37DF8AE271DF61E080E0FD
:1002B0001FDF61E080E01CDF8CE469DF8FE667DF31
:1002C00086E765DF85E663DF61E080E011DF61E0FE
:1002D00080E00EDF61E080E00BDF61E080E008DFBE
:1002E00061E080E005DF83E552DF89E650DF8CE6E0
:1002F0004EDF86E74CDF89E64ADF81E648DF61E0D2
:1003000080E0F6DE61E080E0F3DE8AE240DF48E88C
:1003100052E061E080E058DF41E029E130E088B35D
:10032000842788BB88E893E1F9013197F1F70197B9
:10033000D9F7F5CF6CD008F481E0089594D088F017
:100340009F5790F0B92F9927B751A0F0D1F0660FC1
:10035000771F881F991F1AF0BA95C9F712C0B130DC
:1003600081F09BD0B1E0089598C0672F782F88273F
:10037000B85F39F0B93FCCF3869577956795B3951B
:10038000D9F73EF490958095709561957F4F8F4F8A
:100390009F4F0895E89409C097FB3EF4909580958F
:1003A000709561957F4F8F4F9F4F9923A9F0F92F3B
:1003B00096E9BB279395F695879577956795B795B9
:1003C000F111F8CFFAF4BB0F11F460FF1BC06F5F9F
:1003D0007F4F8F4F9F4F16C0882311F096E911C0B1
:1003E000772321F09EE8872F762F05C0662371F0D2
:1003F00096E8862F70E060E02AF09A95660F771FE6
:10040000881FDAF7880F9695879597F90895990FC1
:100410000008550FAA0BE0E8FEEF16161706E807CE
:10042000F907C0F012161306E407F50798F0621BEF
:10043000730B840B950B39F40A2661F0232B242BC4
:10044000252B21F408950A2609F4A140A6958FEFE3
:10045000811D811D089557FD9058440F551F59F077
:100460005F3F71F04795880F97FB991F61F09F3FA1
:1004700079F087950895121613061406551FF2CFCA
:100480004695F1DF08C0161617061806991FF1CF1A
:1004900086957105610508940895E894BB27662741
:1004A0007727CB0197F90895B2DF08F48FEF08950D
:1004B0000AD080C071D028F076D018F0952309F0CA
:1004C00062C067C0EBCFC7DFA8F39923D9F35523E8
:1004D000C9F3950F50E0551FAA27EE27FF27BB272A
:1004E00000240894679520F4E20FF31FB41F0A1E3E
:1004F000220F331F441FAA1F6695A9F7779530F482
:10050000F30FB41F0A1E121E08F46395330F441F25
:10051000AA1F221F769599F7879520F4B40F0A1E1B
:10052000121E631F440FAA1F221F331F8695A9F7AF
:10053000862F712D602D11249F5750408AF0E1F0D5
:1005400088234AF0EE0FFF1FBB1F661F771F881F0F
:1005500091505040A9F79E3F510570F014C09ECFB6
:100560005F3FECF3983EDCF3869577956795B795FA
:10057000F795E7959F5FC1F7FE2B880F911D969524
:10058000879597F9089597F99F6780E870E060E094
:1005900008959FEF80EC089500240A94161617061C
:1005A00018060906089500240A9412161306140664
:1005B00005060895092E0394000C11F4882352F0C7
:1005C000BB0F40F4BF2B11F460FF04C06F5F7F4F7F
:1005D0008F4F9F4F08950024552704C0080E591FC0
:1005E000880F991F009729F076956795B8F37105E4
:0C05F000B9F7802D952F0895F894FFCFE7
:1005FC000000000000000000002F000000000700B9
:10060C00070000147F147F1400242A7F2A12006232
:10061C0064081323003649552250000005030000DE
:10062C0000001C224100000041221C000014083E66
:10063C0008140008083E0808000000A0600000082C
:10064C000808080800006060000000201008040280
:10065C00003E5149453E0000427F4000004261513E
:10066C004946002141454B31001814127F100027D8
:10067C0045454539003C4A4949300001710905039B
:10068C0000364949493600064949291E00003636CC
:10069C00000000005636000000081422410000142F
:1006AC00141414140000412214080002015109060C
:1006BC0000324959513E007C1211127C007F49498D
:1006CC004936003E41414122007F4141221C007FBE
:1006DC0049494941007F09090901003E4149497ACC
:1006EC00007F0808087F0000417F41000020404146
:1006FC003F01007F08142241007F40404040007FB2
:10070C00020C027F007F0408107F003E4141413EF5
:10071C00007F09090906003E4151215E007F09193D
:10072C0029460046494949310001017F0101003F3A
:10073C004040403F001F2040201F003F4038403FBA
:10074C00006314081463000708700807006151491E
:10075C00454300007F41410000552A552A550000B1
:10076C0041417F000004020102040040404040402F
:10077C00000001020400002054545478007F4844C7
:10078C00443800384444442000384444487F0038FE
:10079C005454541800087E0901020018A4A4A47C27
:1007AC00007F080404780000447D400000408084F1
:1007BC007D00007F102844000000417F4000007C39
:1007CC0004180478007C0804047800384444443845
:1007DC0000FC242424180018242418FC007C080491
:1007EC00040800485454542000043F444020003C6A
:1007FC004040207C001C2040201C003C4030403CF1
:10080C00004428102844001CA0A0A07C0044645480
:0E081C004C441414141414144C4F5645000090
:00000001FF
